:100000000C94F6010C942E020C942E020C942E02E9
:100010000C942E020C942E020C942E020C942E02A0
:100020000C942E020C942E020C94681F0C94372012
:100030000C94481A0C942E020C942E020C942E024E
:100040000C942E020C942E020C942E020C942E0270
:100050000C942E020C94D01A0C942E020C942E02A6
:100060000C942E020C942E020C942E020C942E0250
:100070000C942E020C942E020C942E020C942E0240
:100080000C942E020C942E020C942E020C942E0230
:100090000C942E020C942E020C942E020C942E0220
:1000A0000C942E020C942E020C942E02F104F104F6
:1000B0001D051D058505A305BB06BB06AE05470648
:1000C000580658065117471754179C17A017A01722
:1000D0009C17A017A0177517A0177F178917A017CF
:1000E000A017A017A0179C17A017A0179C17A01760
:1000F0006217A017A01799179917991799179917A9
:1001000099179917991799179E17A0175117441700
:10011000A017A017A017A017A017A017A017A01727
:10012000A017A0179E17A017A0179C17A017971726
:10013000971797179717971797179717971797174F
:100140009E17A420CB20C321CB20C32117213A2105
:10015000C3219121A02135001E001F002000210095
:100160002200230024002500260027002D002E0059
:100170002A0001532B0014001A0008001500170074
:100180001C0018000C00120013002F00300031007A
:100190004B00390004001600070009000A000B009C
:1001A0000D000E000F0033003400280000004E0048
:1001B000E1001D001B0006001900050011001000E1
:1001C000360037003800E500000052002900E0004A
:1001D000E200E30000002C0000000000000000002E
:1001E000E700E6000000500051004F0029003A00EF
:1001F0003B003C003D003E003F004000410042000B
:10020000430044004500010001530100C35CC55C8C
:10021000C45CC75CC65CC95CC85CCB5CCC5CCD5CB8
:10022000CC5C0100010001000100CE5CCF5CD05C21
:10023000D15CD25CD35CD45CD55CD65C010001009F
:1002400001000000010001000100010001000100A7
:100250000100010001000100010001000100000097
:100260000100010001000100010000000100000088
:10027000000000000000010001000000010001007A
:100280000100100362006F006C0073006100360013
:10029000350000000E0346004A004C006100620079
:1002A000730000000403090409023B00020100A0DE
:1002B000FA090400000103010100092111010001F4
:1002C0002240000705810308000109040100010321
:1002D00000000009211101000122B6000705820378
:1002E00020000112010002000000087470010001EA
:1002F000000102000105010902A10185020901A115
:1003000000050919012908150025019508750181C5
:10031000020501093009311581257F950275088193
:100320000609381581257F950175088106050C0A97
:1003300038021581257F950175088106C0C0050129
:100340000980A101850319012AB700150126B7000C
:10035000950175108100C0050C0901A101850419E2
:10036000012AA002150126A002950175108100C086
:1003700005010906A1018506050719E029E7150011
:1003800025019508750181020507190029EF15005F
:10039000250195F0750181020508190129059505CA
:1003A00075019102950175039101C005010906A12E
:1003B00001050719E029E715002501950875018158
:1003C000029501750881010507190029FF1500260E
:1003D000FF00950675088100050819012905950596
:1003E00075019102950175039101C00011241FBE92
:1003F000CFEFDAE0DEBFCDBF04B603FE18C08091B8
:10040000C9029091CA02A091CB02B091CC02873070
:10041000904BA740B04B59F41092C9021092CA02F7
:100420001092CB021092CC02E0E0F8E3099511E0C3
:10043000A0E0B1E0ECEEF4E402C005900D92A0392A
:10044000B107D9F722E0A0E9B1E001C01D92A93CB3
:10045000B207E1F70E94C1120C9474220C940000C0
:10046000879A0C947211CF93C82F0E94030388239C
:1004700029F0C1FF02C08F9A01C08F98CF910895D3
:1004800081E0089581E008950C94420208950C944F
:1004900046021F93CF93DF9300D000D01F92CDB7B9
:1004A000DEB749835A836B833091930189819A81A6
:1004B000311114C0662359F0222349F00E94F80834
:1004C000182F682F89819A810E94A10803C00E9479
:1004D000CC08182F69817A81812F04C00E94F80806
:1004E00069817A810F900F900F900F900F90DF919C
:1004F000CF911F910C942E10FC01262F4081518129
:100500006281738184810C94490281E00895CF93C4
:10051000DF93EC0160E00E947C02BE01DF91CF918D
:100520000C9447020C9430020C94701108950E94B0
:100530004B070E9496022FE78AE196E02150804007
:100540009040E1F700C000000C94F61A0F931F933F
:10055000CF93DF938C0161E00E947C02EC01B80133
:100560000E9444028823F1F1B801CE010E94931841
:100570008823C1F1B801CE010E945715882391F15B
:10058000B801CE010E94EF17882361F1F801828142
:10059000882309F1CB358DE5D807C1F050F4C1159A
:1005A000FCE5DF0781F0CF3DDC45A9F40E942F0E6A
:1005B00019C0CC35EDE5DE0761F0CD35DD4559F4E8
:1005C0000E94720D08C00E9497020CC00E947B0D11
:1005D00002C00E947E0DC801DF91CF911F910F9143
:1005E0000C94400280E0DF91CF911F910F9108950C
:1005F0000E942A1A0C940F030E9412030C94301AC2
:1006000008950C94000381E008950895CF93C82FB6
:100610000E9401038C2F0E943302CF91089580E045
:100620000C9406030E94EF180C9406030E94EF1826
:1006300090919201891721F0809392010C94060306
:100640000895CF93DF93CDB7DEB72B970FB6F8940D
:10065000DEBF0FBECDBF4F83588769877A878B87F0
:1006600061110E94BE0C9E012F5F3F4F86E0F90191
:1006700011928A95E9F785E0FE013796D90101903C
:100680000D928A95E1F789819A814C815D81452B94
:1006900031F09F3F31F491E08F3F19F403C091E0B6
:1006A00001C090E090FF09C049815A816B817C8133
:1006B0008D819E810E94DF0B05C0C9010E948502C9
:1006C0008111F2CF2B960FB6F894DEBF0FBECDBFCF
:1006D000DF91CF910895FC01808191810E943A09B8
:1006E0000895CF93882309F4A9C0C82F8238C1F494
:1006F0000E94EF1881FDA2C069E3809102019091F0
:1007000003010E94E5190E94E00C2FEF80E792E0C0
:10071000215080409040E1F700C0000069E319C01B
:10072000833801F50E94EF1880FD88C063E5809151
:100730000201909103010E94E5190E94E00C2FEF45
:1007400080E792E0215080409040E1F700C0000037
:1007500063E580910201909103010E94F019CF910D
:100760000C94E00C8438C1F40E94EF1882FD66C03E
:1007700067E480910201909103010E94E5190E94B3
:10078000E00C2FEF80E792E0215080409040E1F7AD
:1007900000C0000067E4DDCF8CEF8C0F813AF8F4E5
:1007A0008C2F0E94A617811149C06C2F80910201E5
:1007B000909103010E946519882349F06C2F809164
:1007C0000201909103010E94F0190E94E00C6C2F2D
:1007D00080910201909103010E94E519C0CF80E24F
:1007E0008C0F883048F4C77081E001C0880FCA952B
:1007F000EAF70E94A10CB3CFEBE5EC0FE33040F435
:10080000F0E0E95BFE4F808190E0CF910C942319DA
:10081000E8E5EC0FE73150F4F0E0EE0FFF1FE75E84
:10082000FE4F80819181CF910C943919CD3E30F0EB
:100830008C2F0E944613CF910C941814CF910895D9
:10084000882309F464C0823879F40E94EF1881FF8C
:100850005EC069E380910201909103010E94E51955
:100860000E94E00C69E310C08338B1F40E94EF18D5
:1008700080FF4DC063E580910201909103010E94C9
:10088000E5190E94E00C63E580910201909103015B
:100890000E94F0190C94E00C843879F40E94EF184F
:1008A00082FF35C067E480910201909103010E94AC
:1008B000E5190E94E00C67E4E7CF9CEF980F913AAE
:1008C00010F4682FE1CF90E2980F983050F48770C1
:1008D00091E001C0990F8A95EAF7892F0E94A70C31
:1008E000D9CF9BE5980F933020F480E090E00C94F2
:1008F000231998E5980F973120F480E090E00C944C
:1009000039198D3E20F00E94A1130C9418140895FB
:100910001F93CF93DF93182FEB010E947103209751
:1009200041F08FEC97E00197F1F700C000002197AC
:10093000F6CF812FDF91CF911F910C942004893342
:1009400019F060E070E002C060E570E00C9488048B
:10095000882321F00E94A10C0C94E00C08958823B8
:1009600021F00E94A70C0C94E00C0895CF92DF9226
:10097000EF92FF920F931F93CF93DF937C01D62FBB
:10098000C72FFC011281058102950F700E94970C00
:100990008823B9F01123A9F08C2F807F803421F0B7
:1009A00080E28D0F883068F08091A30282FD09C03B
:1009B00082E00E94400D0E94970C91E0D82ED9262B
:1009C00001C0D12CCC2EC2948FE0C8228C2D90E097
:1009D0008C30910508F0CFC1FC01EA5AFF4F0C940E
:1009E0000B228C2F807FCF70882311F0C295C07F9F
:1009F000112399F0CC2309F4AAC180E28D0F88302D
:100A000010F0D11104C08C2F0E94A10C03C08C2FB8
:100A10000E94B10C0E94E00C9AC18D2F0E9420040C
:100A2000CC2309F4A8C180E28D0F883038F1DD2392
:100A300029F18C2F0E94B70C24C08C2F807FCF709F
:100A4000803211F0C295C07FDD2319F0D130A1F1C1
:100A50003DC08091A30282FF17C0112349F0CC232F
:100A600029F08C2F0E94A10C0E94E00C80E070C144
:100A700080E00E942004CC2309F47DC18C2F0E94C9
:100A8000A70C0E94E00C77C1112371F0002341F004
:100A9000013031F40E94C10C8C2B0E94C90C6BC137
:100AA0000E94C10C8C2B1DC0002319F0013009F4E9
:100AB00062C10E94D60C25C0112321F0063008F037
:100AC0005AC10EC0053008F056C11BC0112361F099
:100AD000002331F0F701858180FF39C18F70858354
:100AE0008C2F0E94A80447C1002359F0D93309F084
:100AF0003FC1FFEF03EF11E0F15000401040E1F77C
:100B000035C18C2F0E94AF0436C18C2F86958695F7
:100B1000837019F0813061F02EC1112321F08D2FE7
:100B20009C2F937002C080E090E00E9423192BC19B
:100B3000112321F08D2F9C2F937002C080E090E054
:100B40000E94391920C18D2F112319F00E944613DC
:100B500002C00E94A1130E94181415C18C2F83702B
:100B600009F047C011110BC12D2F22952695277032
:100B7000220F220F6D2F6F70862F90E0A0E0B0E063
:100B8000022E04C0880F991FAA1FBB1F0A94D2F718
:100B9000D4FF10C04FE050E060E070E004C0440FAC
:100BA000551F661F771F2A95D2F74095509560957F
:100BB000709503C040E050E0BA01C695C695C37079
:100BC0008A019B01082B192B2A2B3B2BC901B80149
:100BD000C23049F058F4C13019F00E94B707CFC0B5
:100BE0000E94A507CCC00E94C907C9C00E94A307E4
:100BF000C6C0112319F08C2F817001C086958823FF
:100C000009F4BDC02D2F229526952770220F220FA3
:100C10006D2F6F70862F90E0A0E0B0E0022E04C030
:100C2000880F991FAA1FBB1F0A94D2F7D4FF10C0C8
:100C30004FE050E060E070E004C0440F551F661FB5
:100C4000771F2A95D2F7409550956095709503C00F
:100C500040E050E0BA01C695C695C3708A019B0179
:100C6000082B192B2A2B3B2BC901B801C23049F0A4
:100C700058F4C13019F00E947C0881C00E946A08B3
:100C80007EC00E948E087BC00E94DD0778C0CF70B6
:100C9000112339F08C2F0E9403088D2F0E94A80485
:100CA0006EC08D2F0E94AF048C2F0E94240867C055
:100CB000D23F21F128F4D03F41F0D13FC1F043C0F1
:100CC000D33F19F1D43F79F03EC0112341F00530F4
:100CD00008F051C08C2F8F710E9449084CC006301B
:100CE00008F049C0F7CF8091A30282FF18C01123FA
:100CF00039F08C2F8F710E9403083DC01123C9F376
:100D00008C2F8F710E94240836C0112329F08C2F5C
:100D10008F710E94EE072FC00E94E9072CC011239B
:100D200049F0CF718C2F0E94030863E08C2F0E9442
:100D3000250D21C081E00E94400D0230E0F082E0EC
:100D40000E94400D18C0112331F0002391F28D2F25
:100D50000E94710310C0002399F2D93349F41FEFA8
:100D600023EF31E0115020403040E1F700C0000097
:100D70008D2F0E94200488EF8C0D843020F40E9477
:100D8000EF180E940603DD20C9F00E94930C80FD3D
:100D900015C0F70112820E948D0C0E940308C70142
:100DA0000E94FF060E948D0CDF91CF911F910F9141
:100DB000FF90EF90DF90CF900C942408DF91CF91BB
:100DC0001F910F91FF90EF90DF90CF9008950F93B8
:100DD0001F93CF93DF93EC01688179818A810E9410
:100DE00045098C010E94A0080E949107B801CE011C
:100DF0000E94B604DF91CF911F910F910895CF9378
:100E0000DF93EC01988189812B813C81232B31F088
:100E10008F3F31F481E09F3F19F403C081E001C0AE
:100E200080E080FD1DC0CE010E94A602811110C08D
:100E30000E94970C8823A1F08A81882389F08091F1
:100E4000A30282FD0DC082E0DF91CF910C94400D92
:100E5000CE010E94E706CE01DF91CF910C9487026C
:100E6000DF91CF91089580E090E00E94231980E007
:100E700090E00E9439190E94BE0C0E94E00C0E9472
:100E800049150C94181480910201909103010E945D
:100E9000FB190C9433070E94AE0C0C9443079295F7
:100EA0009F70963079F010F4925001C09A509230B1
:100EB00068F4803F69F018F4883E40F409C0843F2C
:100EC00029F406C0883E20F0813F11F080E00895AB
:100ED00081E00895FC01808191810E943A090E947D
:100EE0004F070895CF93DF9300D000D01F92CDB766
:100EF000DEB70F900F900F900F900F90DF91CF9172
:100F00000895CF93DF9300D000D000D0CDB7DEB7E7
:100F100026960FB6F894DEBF0FBECDBFDF91CF91FE
:100F20000895089508950C9492070C9493070E94D5
:100F300095076093CA017093CB018093CC01909385
:100F4000CD010C9433070C9497070F931F930091D6
:100F5000CA011091CB012091CC013091CD01602BC1
:100F6000712B822B932B1F910F910C9497070F934A
:100F70001F930091CA011091CB012091CC013091B7
:100F8000CD0160237123822393231F910F910C9431
:100F900097070F931F930091CA011091CB012091E5
:100FA000CC013091CD0160277127822793271F91B3
:100FB0000F910C9497070C9492070E94DB076093A3
:100FC000C6017093C7018093C8019093C9010C9426
:100FD000330760E070E0CB010C94DD070F931F93A3
:100FE00041E050E060E070E08A019B0104C0000F26
:100FF000111F221F331F8A95D2F7C901B8011F9113
:101000000F910C94DD070F931F9341E050E060E0D7
:1010100070E004C0440F551F661F771F8A95D2F7F2
:101020008091C6019091C701A091C801B091C901FA
:101030008A019B01082B192B2A2B3B2BC901B801D4
:101040001F910F910C94DD070F931F9341E050E027
:1010500060E070E004C0440F551F661F771F8A953B
:10106000D2F740955095609570958091C60190910A
:10107000C701A091C801B091C9018A019B01082351
:1010800019232A233B23C901B8011F910F910C9406
:10109000DD070F931F9341E050E060E070E004C073
:1010A000440F551F661F771F8A95D2F78091C6019E
:1010B0009091C701A091C801B091C9018A019B011B
:1010C000082719272A273B27C901B8011F910F912B
:1010D0000C94DD070F931F930091C6011091C70177
:1010E0002091C8013091C901602B712B822B932B69
:1010F0001F910F910C94DD070F931F930091C60170
:101100001091C7012091C8013091C901602371235A
:10111000822393231F910F910C94DD070F931F934C
:101120000091C6011091C7012091C8013091C901F9
:1011300060277127822793271F910F910C94DD0759
:1011400008952FE0929F800D1124E82FE695E695F3
:10115000E695877051E001C0550F8A95EAF785E062
:10116000E89FF0011124EC56FE4F20E030E070E0E3
:101170004081CB01022E02C0969587950A94E2F732
:101180008170819584278523842781932F5F3F4F2A
:101190002530310569F708952FE0929F800D1124C5
:1011A000682F669566956695982F977085E0689F7D
:1011B000B001112440E050E080E0FB01E40FF51F96
:1011C000EC56FE4F208130E0092E02C0369527955F
:1011D0000A94E2F721703327042E01C0220F0A94EB
:1011E000EAF7822B4F5F5F4F4530510531F7089585
:1011F000BF92CF92DF92EF92FF920F931F93CF9304
:10120000DF938C01C090C601D090C701E090C80167
:10121000F090C9018091CA019091CB01A091CC01BD
:10122000B091CD01C82AD92AEA2AFB2ACFE1D0E021
:10123000D701C6010C2E04C0B695A7959795879542
:101240000A94D2F780FD04C0219790F7B12C07C013
:10125000BC2EB8018C2F0E9441100197A9F38B2D51
:10126000DF91CF911F910F91FF90EF90DF90CF9082
:10127000BF900895CF93DF93EC010E94F808BE0160
:101280000E944110DF91CF9108951F93CF93DF9378
:10129000EB0190919301992321F0CB010E943A092F
:1012A00013C0882349F0CB010E94F808182F682F3B
:1012B000CE010E94A10804C0CB010E94CC08182FC7
:1012C000BE01812F0E944110DF91CF911F9108959F
:1012D0001F93CF93DF93C091CE0116E08091CF0191
:1012E000C81799F0D0E01C9FF0011D9FF00D11244C
:1012F000E053FE4F408151816281738184819581E9
:101300000E9481072196C770E9CFDF91CF911F918D
:101310000895409100025091010260910202709183
:10132000030280910402909105020C948107EF92D0
:10133000FF920F931F93CF93DF93809105028295C5
:101340008F7009F065C080910202882309F460C0A3
:101350008091CE01F090CF01109100020091010226
:10136000609103027091040291E01F3F09F090E048
:10137000C0910001D0910101292F96E0E92E8F152F
:1013800009F446C06115710521F00F3F21F030E0EE
:1013900003C031E001C0322F90E030FD36C0E89E3E
:1013A000F001E99EF00D1124DF01A053BE4F11960C
:1013B0003C911197301329C03C91311326C01296ED
:1013C0003C911297311121C013964D915C91149765
:1013D000461B570B4C175D07C0F4809105028F70B8
:1013E000806180930502EB52FE4F80818F70806197
:1013F000808380E092E00E94FF06DF91CF911F91F1
:101400000F91FF90EF900C94680901968770B7CF09
:10141000DF91CF911F910F91FF90EF9008959F92D0
:10142000AF92BF92CF92DF92EF92FF920F931F93F2
:10143000CF93DF93CDB7DEB761970FB6F894DEBFD9
:101440000FBECDBF8C0185E0F801DE011D96019035
:101450000D928A95E1F7D8011296EC9090910002D6
:10146000E09101022091030230910402211531051F
:1014700031F0EF3F31F481E09F3F19F403C081E088
:1014800001C080E0B82FB1709B2E80FD47C1D8010C
:101490004C9111965C9111971396AD90BC90149756
:1014A00080E0C82E82E0D82EF0900202B501621BC7
:1014B000730B2091000130910101FF2009F4D9C084
:1014C000809105026217730708F095C0282F207FCE
:1014D00009F052C05E1313C0491311C0FE2CE11075
:1014E0000EC08F708061809305020E948909C60139
:1014F0000E94FF0680910502F80185834DC1AB284B
:1015000031F05F3F31F481E04F3F19F403C081E0D7
:1015100001C080E080FD03C081E08E2502C080E034
:1015200090E0F82FF170FF2E80FF1CC08091CE015B
:101530002091CF0136E0821709F40BC190E0389F6B
:10154000F001399FF00D1124E053FE4F61815613D5
:1015500006C06081461303C06281E61203C0019693
:101560008770E9CFFE2CEE2009F416C180910502A8
:1015700081608093050254C05E1306C0491304C005
:10158000E11002C0F80199C0C8010E946A078823CF
:1015900061F1EE2051F120910502822F82958F702A
:1015A00090E0029774F08091000290910102988778
:1015B0008F831986BB86AA862C87CE0107960E9448
:1015C000FF0686E0F801A0E0B2E001900D928A9556
:1015D000E1F70E9497090E9489090AC05E1711F17C
:1015E000C8010E946A0781112CC0C8010E94FF0631
:1015F000FF24F394D1C0282F207F81F77A2DB98A58
:10160000A88A6E2D89890E94720780E092E00E946C
:10161000FF0686E0D6011D928A95E9F70E948909A6
:10162000F12CBAC04913DCCFE110DACFF801858381
:10163000C8010E94FF0686E0D6011D928A95E9F74F
:10164000ABC0EE2091F220910502822F82958F701F
:1016500090E002970CF4B5CF8091000290910102C6
:101660009A8389831B82BD82AC822E83CE01019630
:10167000A6CF6217730708F044C0FE2CEE2009F4D1
:10168000B4CF5E1330C049132EC02091050220FD57
:1016900021C0822F82958F70482F50E0411551054F
:1016A000C9F0F80125834F30510541F08F5F982F25
:1016B0009295907F822F8F70892B8583C8010E941D
:1016C000FF0686E0F801A0E0B2E001900D928A9555
:1016D000E1F73CC086E0F801A0E0B2E001900D9295
:1016E0008A95E1F759C0C8010E946A07811169CF44
:1016F00080910502816080930502C8010E94FF0667
:101700004BC07A2DB98AA88A6E2D89890E947207EA
:1017100086E0D6011D928A95E9F718C0EE2009F4FB
:1017200064CFC8010E946A07F82E882309F45DCFB0
:1017300086E0F801A0E0B2E001900D928A95E1F711
:1017400080E092E00E946B030E9497090E94890941
:1017500023C04D875E878D859E850E943A09292F7B
:1017600022952F70223028F49F7039F0811105C026
:101770000BC0243028F49F7049F4805E883020F03C
:10178000C8010E94FF069F2CF92C06C0D8011596AF
:101790009C91907F91F7F8CF8F2D61960FB6F894BA
:1017A000DEBF0FBECDBFDF91CF911F910F91FF9094
:1017B000EF90DF90CF90BF90AF909F9008951F93D0
:1017C000CF93DF93CDB7DEB72C970FB6F894DEBF7B
:1017D0000FBECDBF4F83588769877A878B879C87D9
:1017E000CE0107960E940F0A8823D1F09F81888539
:1017F0002A853B85232B31F08F3F31F481E09F3FD9
:1018000019F403C081E001C080E080FD47C04F8132
:10181000588569857A858B859C850E9481073EC0A5
:1018200086E0FE013796DE01119601900D928A95B1
:10183000E1F7FF81E8856A857B856115710531F0E7
:10184000EF3F31F481E0FF3F19F403C081E001C0B4
:1018500080E080FD23C02091CF0130E0C9010196D6
:10186000877099274091CE0150E084179507F1F1D8
:10187000F983EA837D836C8396E0929FD001939FE6
:10188000B00D1124A053BE4FFE01319601900D9270
:101890009A95E1F78093CF010E94680916E0809144
:1018A000CE019091CF01891771F1189FC0011124C9
:1018B00080539E4F0E940F0A882329F1E091CE01A8
:1018C0001E9FF0011124E053FE4F4081518162813F
:1018D0007381848195810E9481078091CE0190E07F
:1018E0000196877099278093CE01D9CF0E944B072C
:1018F0001092CF011092CE01E0E0F2E086E0DF012D
:101900001D928A95E9F72C960FB6F894DEBF0FBEAC
:10191000CDBFDF91CF911F910895809126028595CB
:1019200085958595089580912602877008959091F8
:101930002602977081E009F480E0089580914902C1
:10194000089590914902892B8093490208958095CA
:101950009091490289238093490208951092490287
:10196000089590914802892B8093480208958095AC
:10197000909148028923809348020895109248026A
:10198000089580912702089508950C94C40C0C9436
:10199000C50C9091A30292FD08C090912702981760
:1019A00021F0809327020C94C70C089580912702A0
:1019B000882329F01092270280E00C94C70C089528
:1019C000CF93DF93E0910201F091030180914902EE
:1019D0008083E0910201F09103019081809148029F
:1019E000892B808380912702882381F0E091020176
:1019F000F09103019081892B808380910201909165
:101A000003010E944F1981110E94D60CC09102015E
:101A1000D091030140E250E066E072E0CE010E9406
:101A20002522892B69F080E2FE01A6E0B2E0019058
:101A30000D928A95E1F7CE01DF91CF910C94FB18BE
:101A4000DF91CF9108950C94C40C9091A30292FD64
:101A500010C098E0899F90011124262B2093260224
:101A60000E940308809126028595859585950C94A2
:101A7000230D0C9403081092260280E00C94230D91
:101A8000209126028095822380932602982F9770BA
:101A900099F430E0482F082E000C550B2417350719
:101AA00059F09091A30292FD07C085958595859583
:101AB0000E9424080C943B0D08959091A30292FB80
:101AC000222720F9281769F080FB92F99093A3024E
:101AD0008091A2029091A3020E94AB0D82E00C942F
:101AE000400D08958091A30282FB882780F991E040
:101AF00089270C945D0D81E00C945D0D80E00C94C1
:101B00005D0D6FEF7FEF80E090E00C945E2280E04F
:101B100090E00E943A2221E0893E9E4F09F020E0A9
:101B2000822F089582E090E00C94322283E090E0CE
:101B30000C943222CF9384E090E00E943222C82F8E
:101B400082E290E00E9432222C2F30E0A901582B33
:101B5000CA01CF910895CF93C92F682F84E090E0F8
:101B60000E9440226C2F82E290E0CF910C944022A0
:101B7000AB01BC018FE090E00C945222AB01BC01A0
:101B800083E190E00C94522260E070E0CB010C9471
:101B9000BE0D60E070E0CB010E94B80D0C94C40D46
:101BA00069EE7EEF80E090E00E945E2260E082E0DD
:101BB00090E00E94402260E083E090E00E9440229A
:101BC0001092CA011092CB011092CC011092CD015B
:101BD00060E084E090E00E94402260E082E290E0D9
:101BE0000E94402260E085E090E00E94402260E098
:101BF00086E090E00E9440226FEF87E090E00E9434
:101C0000402240E050E0BA0188E090E00E94522279
:101C100060E08DE090E00E94402240E050E0BA0198
:101C200088E190E00E94522260E087E190E00E940B
:101C3000402240E050E0BA018CE190E00E94522244
:101C400060E070E080E290E00E945E2240E050E0C0
:101C5000BA0188E190E00E9452220C94C90D0C94C4
:101C6000D00D682F8EE090E00C9440220E94B51AAF
:101C7000609358027093590280935A0290935B02CA
:101C800060935402709355028093560290935702CA
:101C9000089585B7806885BF85B7806885BF08953A
:101CA00081E008950C94500E08950C94540E0C94F9
:101CB000540E0C94570E0C94540E0C945B0E0C9412
:101CC000540E0E94490E8DE191E10E94E5180E9498
:101CD0005F0E0C945D0E0E94550E0C94540E0E94E3
:101CE00037110C9405030E94A01A0E941A120E9438
:101CF0006F0E0C94590E5F926F927F928F929F920B
:101D0000AF92BF92CF92DF92EF92FF920F931F9309
:101D1000CF93DF93CDB7DEB72A970FB6F894DEBF27
:101D20000FBECDBF0E942F12C82E81110E94360E09
:101D30003AE4832E32E0932E00E010E0502E802F04
:101D40000E945B115C01F401619071904F01682663
:101D5000792661147104B1F40F5F1F4F053011052E
:101D600069F78FEF89838A831B820E94A91A816099
:101D7000782F9D838C8349815A816B818D810E944C
:101D800021033AC080915C0281FD0E946411D12C34
:101D9000EE24E394F12CC3018E219F21892B29F19C
:101DA0000E94520E8823A9F0DE825F82AE20BF20FF
:101DB00081E0AB2809F480E088870E94A91A81603D
:101DC000782F9A8789874E815F8168858A850E94EE
:101DD0002103000F111FF801E65BFD4F8081918107
:101DE000E826F926F182E08207C0D394EE0CFF1CAE
:101DF000FFE0DF12D0CFB0CF81E0C11001C080E0A2
:101E00002A960FB6F894DEBF0FBECDBFDF91CF91FB
:101E10001F910F91FF90EF90DF90CF90BF90AF9008
:101E20009F908F907F906F905F9008950E947B0E9F
:101E30000E9436140C941603CF93DF930E94461031
:101E4000EC01811521E5920708F045C0811530E5C8
:101E5000930708F094C0883E910528F5803E9105CF
:101E600008F0F8C0883A910570F4853A910508F0B9
:101E70007CC08130910509F475C008F4E8C004976E
:101E800008F0E8C0E4C08F3B910508F0E0C0C85AF4
:101E9000D0E0CC0FDD1FC65BDE4F0990D881C02D8E
:101EA000CE019464D8C0811540E2940758F481159E
:101EB00051E0950708F0CEC08D3E910508F4C7C0EB
:101EC0009065C9C0C11580E4D80708F4C0C0DF70B0
:101ED000CE01906AC0C0811525E59207A8F481154E
:101EE00034E5930708F095C0811543E5940708F0A1
:101EF0007BC0811552E5950708F061C0D82FCC272B
:101F0000CE01816F906AA7C0C11589E5D807A0F4FA
:101F1000C11528E5D20708F082C0C11536E5D30700
:101F200008F095C08C2F0E94DA108F7190E0D82FA6
:101F3000CC27CE0190628FC0C1154AE5D40708F4C2
:101F400074C0CE0190568115904208F080C08D2F4C
:101F50008F710E94DA10DD27D0628F71AE01582B8D
:101F6000CA0179C081E090E076C0C55AD0E0C85877
:101F7000DE4F8881C82FD0E0CE0190646CC074E041
:101F8000969587957A95E1F7282F23703C2F33702B
:101F900081E090E002C0880F991F3A95E2F79C68B3
:101FA000AC01522B9A019C2F9F709695969550E20A
:101FB000959FE0011124C9018C2B9D2B4CC083708F
:101FC000992721E030E002C0220F331F8A95E2F703
:101FD0009C2F9695969580E2989FE0011124C22B44
:101FE000D32BCE019C6837C08370992721E030E065
:101FF00002C0220F331F8A95E2F79C2F9695969583
:1020000040E2949FE0011124C22BD32BCE019A68A9
:1020100022C0D82FCC27CE01846F906A1CC0DC2F41
:10202000CC27CE01806F906A16C08C2F8F700E94D3
:10203000DA1094E0D695C7959A95E1F7CF70D0E085
:10204000DC2FCC27D0699E01282BC90104C080E079
:1020500090E001C0CE01DF91CF9108952BE4829FE3
:10206000C0011124FC012FE0729FE00DF11D11242D
:10207000E60FF11DEE0FFF1FEA5AFE4F8591949176
:1020800008950E942E100E941C0F08958238910519
:1020900069F1B0F48133910509F46DC048F48932D7
:1020A000910509F463C08A32910509F469C0089565
:1020B0008533910509F455C089339105B9F0089528
:1020C000833E910569F138F4803E9105B1F0823E7E
:1020D000910509F10895863E9105A9F1873E910584
:1020E000B9F1843E910509F064C023C02091A20299
:1020F00020FD4FC021FD4DC008958091A20280FDBA
:1021000044C08091A30280FF44C08091A20284FD5C
:1021100042C083EE4DC08091A20282FF38C0F5CF4D
:102120008091A20282FD33C08091A30280FD31C064
:10213000ECCF8091A30281FF32C08091A20284FD86
:102140002AC087EE35C08091A20283FF26C0F5CF5A
:102150008091A20283FD21C08091A30281FD1FC056
:10216000ECCF8091A20285FD1CC01DC08091A2020F
:1021700085FD19C016C08091A20286FD16C017C049
:102180008091A20286FD13C010C089E311C082EEC7
:102190000FC080EE0DC080E00BC086EE09C084EE5B
:1021A00007C089E205C085E303C08AE201C081E37C
:1021B00090E008959091A20292FF0DC0282F2871FF
:1021C000283019F4877F846006C0282F24712430BA
:1021D00011F48B7F886093FF0DC0282F2871283160
:1021E00019F4877E846106C0282F2471243111F4EC
:1021F0008B7E88612091A30220FF0DC0382F38719B
:10220000383019F4877F816006C0382F3171313042
:1022100011F48E7F886021FF0DC0282F287128318E
:1022200019F4877E816106C0282F2171213111F4B4
:102230008E7E886194FD877E089580E008950C94D9
:10224000810D0E942F128FE19EE40197F1F700C0EB
:1022500000000E942F1280E00E945B1180FF04C0EA
:102260000E941F110C94F61A08950C9421110E94DB
:10227000870D811102C00E942F0E0E94920D809343
:102280005C020E949A0D9093A3028093A2020E9486
:1022900035110E94960D682F70E080E090E00E945A
:1022A000A3076091C6017091C7018091C801909108
:1022B000C9010C94DB07E82FF0E0EE0FFF1FE25599
:1022C000FD4F808191810895089580E58A95F1F709
:1022D000089500C008950C94651108950C946D1133
:1022E0000C946E110C946D11F894E82FE295EF7038
:1022F000F0E031A1282F2F7081E090E001C0880F1D
:102300002A95EAF7982F9095932391A392A1892B70
:1023100082A3789408950F931F93CF93DF93CAE815
:10232000D1E089918F3F11F00E94741181E0CF3884
:10233000D807B9F7CBE7D1E00AE811E089918F3FE0
:1023400011F00E9474110C171D07C1F7DF91CF9196
:102350001F910F910895BF92CF92DF92EF92FF925B
:102360000F931F93CF93DF938C01C62FD0E0CE0144
:1023700086579E4F6C01FC0190819F3F09F450C02D
:10238000B62EF894E92FE295EF70F0E081A19F70EE
:1023900021E030E001C0220F9A95EAF7822B81A359
:1023A00082A12095282322A378940E946911EBE74B
:1023B000F1E04AE851E021E030E0E12CF12C6191BC
:1023C0006F3F89F0A62FA295AF70B0E090968C91E8
:1023D00090E06F7002C0959587956A95E2F780FD51
:1023E00002C0C90102C080E090E0E82AF92A220F69
:1023F000331F4E175F0719F7F60180818F3F11F0E9
:102400000E94741161E0E114F10409F460E08B2D85
:102410000E946B11CC0FDD1FC00FD11FF982E88223
:10242000DF91CF911F910F91FF90EF90DF90CF90B0
:10243000BF9008950E948B118AE0EEEAF2E0DF017E
:10244000982F1D929A95E9F7E4EAF2E0DF011D92D8
:102450008A95E9F785E00E947A120C949202FF9225
:102460000F931F93CF93DF93CDB7DEB72A970FB6A5
:10247000F894DEBF0FBECDBF8E010F5F1F4F8AE005
:10248000F80111928A95E9F7F12C6F2DC8010E948D
:10249000AB11F394F5E0FF12F8CF4AE050E0B80139
:1024A00084EA92E00E942522FF24F394009709F425
:1024B000F12C892B41F08AE0F801A4EAB2E0019006
:1024C0000D928A95E1F72F2D45E06EEA72E084EADD
:1024D00092E00E947B120E9494028F2D2A960FB6E2
:1024E000F894DEBF0FBECDBFDF91CF911F910F914A
:1024F000FF9008950895FF920F931F93CF93DF935A
:10250000F82E092F162FD72FC42F222349F081E050
:1025100080935F020E94A91A90935E0280935D02ED
:1025200080915F028823D9F080915D0290915E02D4
:102530000E94C11A059798F0EF2DF02FA12FBD2F03
:1025400080E090E04C2F50E08417950734F42191FF
:1025500031912D933D930196F7CF10925F02DF9159
:10256000CF911F910F91FF9008950E94C11C0E946E
:10257000730E0C94CD1C0E94D11C0E94160F0C945B
:10258000EB1C0E94471A0E94A81C0E94610E0E9428
:10259000B5120E94BB120E946B0EFBCF80916602A7
:1025A00080FF06C06091090170E0660F771F26C0AA
:1025B00081FF04C06091090184E005C082FF07C06B
:1025C0006091090188E0689FB001112417C09091C3
:1025D00065029923D1F060910801961788F7209140
:1025E000090188E0289F90011124929FA001939FE8
:1025F000500D112470E0CA010E94F7216038710566
:1026000040F46115710519F406C068E070E0862F8A
:1026100008958FE7089581E008958091660280FF14
:1026200008C06091050170E075956795759567958F
:1026300021C081FF06C06091050170E07595679526
:1026400019C082FF04C06091050170E010C0909134
:102650006402992399F0609104019617A0F7809184
:102660000501899FC001112470E00E94F7216038A4
:10267000710540F46115710519F406C061E070E060
:10268000862F08958FE7089581E008958D3E21F407
:102690000E94CE12819504C08E3E29F40E94CE1273
:1026A00080936A0208958F3E21F40E94CE12819594
:1026B00004C0803F29F40E94CE12809369020895DD
:1026C000893F19F40E940D1305C08A3F31F40E941E
:1026D0000D13819580936B0208958B3F21F40E9426
:1026E0000D13819504C08C3F29F40E940D13809333
:1026F0006C0208959FE0980F983078F421E030E064
:10270000A90102C0440F551F9A95E2F7CA019091A2
:102710006802892B8093680208958D3F21F480918F
:10272000660281600BC08E3F21F480916602826058
:1027300005C08F3F29F48091660284608093660211
:1027400008958D3E39F490916A0297FF35C010923A
:102750006A0259C08E3E29F490916A021916BCF3A0
:102760002BC0909169028F3E29F497FF25C01092EB
:10277000690249C0803F19F41916CCF31DC090912D
:102780006B02893F29F41916BCF410926B023BC00E
:102790008A3F19F497FF10C0F8CF8B3F39F490911E
:1027A0006C0297FF09C010926C022DC08C3F21F47F
:1027B00090916C021916BCF39FE0980F983080F44A
:1027C00021E030E0A90102C0440F551F9A95E2F7BD
:1027D000CA0180959091680289238093680213C092
:1027E0008D3F21F4809166028E7F0BC08E3F21F4D5
:1027F000809166028D7F05C08F3F29F4809166022B
:102800008B7F8093660280916902811106C080915E
:102810006A02811102C01092650280916B028111DF
:1028200006C080916C02811102C01092640208956A
:102830000E94A91A20916902211104C020916A0204
:10284000222321F0909363028093620220916B0215
:10285000211104C020916C02222321F09093610287
:102860008093600287E692E00C941519EF92FF9234
:102870000F931F93CF93DF9300D000D000D0CDB73C
:10288000DEB786E0E7E6F2E0DE01119601900D92F8
:102890008A95E1F7E0906902F0906A0200916B027C
:1028A00010916C021092690210926A0210926B02EF
:1028B00010926C02E11003C0FF2009F45DC080910A
:1028C0006202909163020E94C11AAC01909165026C
:1028D000992339F020910A0130E02417350758F088
:1028E0004BC020910B018AE0289F900111242417EE
:1028F000350718F041C09F3F19F09F5F9093650224
:10290000EE2061F00E94CE121E1414F09FEF01C061
:1029100091E0989F902D112490936902FF2061F01F
:102920000E94CE121F1414F09FEF01C091E0989FF7
:10293000902D112490936A02309169023323E1F0C3
:1029400020916A022223C1F045EB3403C001112417
:10295000992319F09093690203C081E08093690282
:1029600035EB2303C0011124992319F090936A02D7
:1029700003C081E080936A02011103C0112309F4AE
:102980005DC080916002909161020E94C11AAC0109
:1029900090916402992339F02091060130E02417C8
:1029A000350758F04BC0209107018AE0289F90011D
:1029B00011242417350718F041C09F3F19F09F5F7D
:1029C00090936402002361F00E940D13101614F01E
:1029D0009FEF01C091E0989F902D112490936B027E
:1029E000112361F00E940D13111614F09FEF01C026
:1029F00091E0989F902D112490936C0230916B027E
:102A00003323E1F020916C022223C1F045EB340323
:102A1000C0011124992319F090936B0203C081E047
:102A200080936B0235EB2303C0011124992319F025
:102A300090936C0203C081E080936C0280916902E4
:102A400081110BC080916A02811107C080916B02D5
:102A5000811103C080916C0281110E941814EB82D5
:102A6000FC820D831E8386E0FE013196A7E6B2E06C
:102A700001900D928A95E1F726960FB6F894DEBF85
:102A80000FBECDBFDF91CF911F910F91FF90EF90BF
:102A90000895E7E6F2E086E0DF011D928A95E9F706
:102AA0001092650210926402109266020895CF930C
:102AB000DF93EC01FB018281882309F43CC1C4301F
:102AC000FDE5DF0760F4CB3F9CE5D90788F49E0164
:102AD00022503C452431310508F02EC109C0C236D0
:102AE000EDE5DE0729F0C63AFDE5DF0709F024C170
:102AF0000E949A0D9093A3028093A202C1318CE5AB
:102B0000D80709F4C6C008F042C0C930ECE5DE07BA
:102B100009F49BC000F5C5308CE5D80709F485C0E1
:102B200078F4C330ECE5DE0709F478C008F07AC029
:102B3000C230DC4509F0F5C08091A2028160EFC08F
:102B4000C7309CE5D90709F478C008F07AC08091B5
:102B5000A2028061E4C0CD30FCE5DF0709F487C044
:102B600058F4CB309CE5D90709F479C008F07BC054
:102B70008091A20288606FC0CF30FCE5DF0709F4C6
:102B800080C008F082C08091A202877FC8C0CE3F7B
:102B90009CE5D90709F471C000F5C531FCE5DF07F4
:102BA00009F485C068F4C3319CE5D90709F475C000
:102BB00008F095C00E944B078091A2028F77AFC0AA
:102BC000CC3FFCE5DF07A9F108F054C0CB3FDC4562
:102BD00009F0A7C08091A30240C0C230EDE5DE0736
:102BE00009F489C058F4C1158DE5D80709F45AC015
:102BF00008F069C08091A30282602FC0C236EDE563
:102C0000DE0709F47CC0C63AFDE5DF0709F481C0A0
:102C1000C330DD4509F085C080E06EC08091A2021E
:102C200082607DC08091A20216C08091A20288605D
:102C300076C08091A30282604FC08091A202806220
:102C40006EC08091A20280646AC00E944B0780918E
:102C5000A202806864C0846062C081603DC08091CF
:102C6000A2028E7F5CC08091A2028D7F58C08091AD
:102C7000A20216C08091A30218C08091A3028D7F8A
:102C80002BC08091A2028F7E4AC08091A2028F7DCC
:102C900046C08091A2028F7B42C08091A202877FB2
:102CA0008B7F3DC08091A3028D7F8E7F15C0809168
:102CB000A20282FB222720F991E0922790FB82F961
:102CC00090FB83F92CC08091A302982F909591706E
:102CD0008E7F892B90FB81F98093A30222C00E94F2
:102CE0004B078091A20287FB222720F991E09227CF
:102CF00090FB87F914C081E00E94310E12C08091D0
:102D0000A20284FB222720F991E0922790FB84F90C
:102D100006C08091A202982F909590FB80F9809335
:102D2000A2028091A2029091A3020E94AB0D0E9488
:102D30004B0780E001C081E0DF91CF910895893297
:102D400089F1F0F4843171F1B0F4873009F077C083
:102D500081E080930B0184E180930A018AE08093F3
:102D600009018EE18093080188E08093050188E2E3
:102D70008093040164C092EE980F9A30F0F05FC027
:102D8000803509F444C028F48F3409F058C08AE033
:102D90003FC0813529F0823509F051C081E038C04B
:102DA0008FEF36C080916F02882379F110926F0205
:102DB00010926E0210926D0242C08D5180936F028C
:102DC000833099F038F4813069F08230D9F48AE0A8
:102DD00091E00DC0853099F078F0863099F484E068
:102DE00091E005C08BE091E002C089E091E0909312
:102DF0006E0280936D0223C088E091E0F8CF85E0F9
:102E000091E0F5CF10926F021AC080E0089586EF2E
:102E1000E0916D02F0916E02309789F02081082ECA
:102E2000000C990B820F911D8F3F910519F014F042
:102E30008FEF04C097FF02C0108201C0808381E041
:102E400008950F931F9341E050E060E070E08A0125
:102E50009B0104C0000F111F221F331F8A95D2F758
:102E6000C901B8010E94A3071F910F910C944B0751
:102E7000482F50E0FA013597EF33F10508F060C0B4
:102E8000EE59FF4F0C940B220E942F0E55C08091DB
:102E90005C02817F8E7F80935C0281E08093700270
:102EA00008950E94970248C080915C02982F9095E7
:102EB000917090FB80F980935C0291113DC0897FF5
:102EC000877F10C080915C0281FB222720F991E06E
:102ED000922790FB81F980935C02992369F180919C
:102EE0005C02816080935C0227C080915C0282FB5F
:102EF000222720F991E0922790FB82F9ECCF809174
:102F00005C0283FB222720F991E0922790FB83F952
:102F1000E2CF0E944B078091A20287FB222720F973
:102F200091E0922790FB87F98093A20205C0895314
:102F300001C08D510E94211781E0089580E0FACFF1
:102F400080E0089580E008950C94A217CF93C82FD5
:102F500080917002813069F038F08230C1F58C2F99
:102F60000E949F1681E039C00E949E0C823289F532
:102F700004C00E949E0C823261F48C2F0E94A41720
:102F8000811104C08C2F0E9438171FC081E090E08F
:102F90001CC08C2F0E94A217811116C0C43189F069
:102FA00058F4CB3089F0C031B1F482E080937002E4
:102FB00088E30E949F1608C0C93219F0C83321F077
:102FC0000AC01092700207C081E0817006C01092A2
:102FD000700280E002C080E0F8CFCF910895CF93D7
:102FE000DF9386319C4541F5EB010E949E0C982FA2
:102FF0008A812091020130910301882379F09A7A25
:1030000081E009F480E080937102911102C069E2CD
:1030100001C065E3C9010E94E5190AC080917102EF
:10302000811102C069E201C065E3C9010E94F01983
:103030000E94E00C80E001C081E0DF91CF91089513
:103040000F931F93CF93DF93C42FD22FFC01828164
:103050008823C9F0409374020E94A91A90937302C6
:103060008093720280E28C0F883008F057C0C770DE
:1030700081E001C0880FCA95EAF7DF91CF911F91D7
:103080000F910C94A80480917402481330C0809171
:103090007202909173020E94C11A883C910538F522
:1030A00010E21D0FCD17B9F080E28C0F883040F48C
:1030B000C77081E001C0880FCA95EAF70E94AF048B
:1030C000183028F581E09D2F977001C0880F9A95E0
:1030D000EAF70E94A804802F0E949F041830F0F4A1
:1030E000D77081E001C0880FDA95EAF70AC080E264
:1030F0008C0F883098F4C77081E001C0880FCA95A2
:10310000EAF7DF91CF911F910F910C94AF04802FBC
:10311000DF91CF911F910F910C949F04DF91CF917C
:103120001F910F9108950F939C01CB01243F4CE513
:10313000340731F188F4293DFCE53F07D9F02A3DF9
:103140004CE5340779F1283D3C45A9F506E221EE2E
:1031500041EE68ED7CE52BC0263FFCE53F07E1F042
:10316000A8F0273F3C4539F507E225EE46EE67EF2C
:103170007CE51DC007E225EE45EE69ED7CE517C054
:1031800006E221EE40EE64EF7CE511C007E225EE99
:1031900044EE65EF7CE50BC006E221EE42EE66EF01
:1031A0007CE505C008E221E045EE6AED7CE50E9481
:1031B000201880E008C0FC018281882319F0109259
:1031C000740201C081E00F91089590939101809362
:1031D0009001089590937A02809379020895E09186
:1031E0007902F0917A02309721F00190F081E02D80
:1031F000099480E00895E0917902F0917A02309785
:1032000099F020911801222359F02091A20227FF62
:1032100007C0DC012C9111962C93119726E02C937A
:103220000280F381E02D09940895E0917902F091F4
:103230007A02309739F022E0DC012C930480F5818A
:10324000E02D099408952091770230917802281793
:10325000390771F09093780280937702E0917902B8
:10326000F0917A02309721F00680F781E02D0994E1
:10327000089520917502309176022817390771F070
:103280009093760280937502E0917902F0917A0230
:10329000309721F00084F185E02D09940895FC0118
:1032A000329680911801882331F08091A20287FF25
:1032B00002C09EE101C096E080E0915028F021918B
:1032C0002223D9F38F5FF9CF0895662351F120911E
:1032D00018012223E9F02091A20227FF19C0462FEE
:1032E0004695469546954E31E0F4677021E030E012
:1032F00002C0220F331F6A95E2F7FC01E40FF11DB3
:10330000828190E02823392381E0232B69F409C0CE
:10331000FC01329608962191621729F0E817F90707
:10332000D1F780E0089581E008959C01FC01329678
:103330009FEF80E04191461789F09F3F19F44111BA
:1033400001C0982F8F5F8630A9F79F3F39F0F901B0
:10335000E90FF11D97FDFA956283089508959C0188
:103360002A5F3F4FFC014281461301C01282019641
:1033700082179307B9F70895262F26952695269547
:103380002E3168F4FC01E20FF11D677021E030E09E
:1033900001C0220F6A95EAF78281282B22830895C3
:1033A000262F2695269526952E3170F4FC01E20FE6
:1033B000F11D677021E030E001C0220F6A95EAF745
:1033C00020958281282322830895209118012223A9
:1033D00029F02091A20227FD0C94BC190C94951998
:1033E00020911801222329F02091A20227FD0C949C
:1033F000D0190C94AF1920911801FC0132962223A8
:1034000031F08091A20287FF02C08EE101C086E008
:10341000DF011D928A95E9F7089508950C940D1A1D
:1034200083E080937B020C940E1A811102C081E02C
:1034300001C082E080937B020C940E1A0C94151A42
:1034400081E080937B020C940E1A0C94201A08954C
:103450000C94271A0C94281A0C94271A0C94271AE7
:103460000C94271ACF930E942E1A0E942F120E94AA
:103470002C1AC0E08C2F0E945B11892B29F4CF5F9E
:10348000C530C1F780E001C081E0CF910895089573
:103490001F920F920FB60F9211248F939F93AF93A9
:1034A000BF9380917C02811113C08091B8029091EA
:1034B000B902A091BA02B091BB024196A11DB11D03
:1034C0008093B8029093B902A093BA02B093BB0262
:1034D000BF91AF919F918F910F900FBE0F901F9052
:1034E00018958091C002843031F10E94F802109248
:1034F0007C0220E488E190E00FB6F894A8958093D0
:1035000060000FBE2093600083B7817F846083BF1B
:1035100083B7816083BF7894889583B78E7F83BF9C
:103520000FB6F894A8958091600088618093600040
:10353000109260000FBE08950E944B070C94FC028D
:1035400082E084BD93E095BD9DE797BD80936E00BA
:1035500008952FB7F8948091B8029091B902A09184
:10356000BA02B091BB022FBF08952FB7F8946091B3
:10357000B8027091B9028091BA029091BB022FBF3C
:1035800008959C014FB7F8948091B8029091B902C8
:10359000A091BA02B091BB024FBF821B930B08955A
:1035A00078941F920F920FB60F9211248F939F93CE
:1035B000AF93BF938091B8029091B902A091BA02E3
:1035C000B091BB020196A11DB11D8093B8029093EA
:1035D000B902A093BA02B093BB02BF91AF919F9181
:1035E0008F910F900FBE0F901F90189581E08093E0
:1035F000E00080E28093D8001092C9008FE097E24B
:103600000197F1F700C0000087E090EBDC018093A8
:10361000C9029093CA02A093CB02B093CC029CE063
:1036200088E10FB6F894A895809360000FBE909340
:103630006000FFCF8091A0020895089522E02093BA
:10364000E9002FEF3091E800215035FD06C03AE641
:103650003A95F1F700C02111F5CF2091E80025FF40
:103660000BC040E050E066E070E00E945C1D80917D
:10367000E8008E778093E8000895CF93DF93209140
:103680001801222339F02091A20227FF03C060E233
:1036900022E002C068E021E02093E9002FEF3091A2
:1036A000E800215035FD06C03AE63A95F1F700C032
:1036B0002111F5CF2091E80025FF1DC0EC0180917C
:1036C0001801811105C040E050E068E070E003C0DF
:1036D00070E040E050E0CE010E945C1D8091E80067
:1036E0008E778093E80080E2FE01A0E8B2E00190CE
:1036F0000D928A95E1F7DF91CF91089580937D0235
:1037000070937F0260937E028091C002843001F545
:1037100082E08093E9008FEF9091E800815095FD61
:1037200006C09AE69A95F1F700C08111F5CF809115
:10373000E80085FF0DC040E050E063E070E08DE7F9
:1037400092E00E945C1D8091E8008E778093E800F3
:103750000895BC0184E00C947E1BBC0183E00C94B2
:103760007E1B8091BF02811109C00E94ED1E0E9444
:103770004A1F8091E20084608093E20008951092D5
:10378000BF0208950C94251A6091BC0281E061117A
:1037900001C080E00C94101A9091C00281E0943036
:1037A00009F080E06091BC020C94151A42E061ECD3
:1037B00081E00E94661E42E261EC82E00E94661E89
:1037C0009091C00281E0943009F080E06091BC02E9
:1037D0000C941E1A8091C202833009F461C030F447
:1037E000813071F0823009F49AC008958A3009F46A
:1037F00086C08B3009F46CC0893009F0A8C020C0A5
:103800008091C102813A09F0A2C08091E800877FCF
:103810008093E8008091C5029091C602892B21F423
:1038200060E280E892E003C060E080E090E070E059
:103830000E94A71D8091E8008B778093E80008958F
:103840008091C102813209F082C08091C5029091BD
:10385000C602029708F07BC08091E800877F8093C2
:10386000E8008091E80082FD05C08091C0028111CE
:10387000F8CF6DC02091F3008091F20090E0922B80
:10388000029731F48091F100813011F0863021F4FB
:103890008091F1008093A0028091E8008B7753C063
:1038A0008091C102813A09F052C08091C502909185
:1038B000C602892B09F04BC08091E800877F809376
:1038C000E8008091E80080FFFCCF8091180136C0AD
:1038D0008091C1028132D9F58091C5029091C602D2
:1038E000892BA9F58091E800877F8093E8000E94EA
:1038F0009B1E8091C302809318010C944B0780910A
:10390000C102813221F58091E800877F8093E80031
:103910000E949B1E8091C4028093A1020895809111
:10392000C102813AA1F48091E800877F8093E8008A
:103930008091E80080FFFCCF8091A1028093F1008C
:103940008091E8008E778093E8000C949B1E089588
:1039500084B7877F84BF0FB6F894A89580916000E4
:10396000886180936000109260000FBE90E080E854
:103970000FB6F89480936100909361000FBE0C9491
:10398000201A0E94ED1E0E944A1FE2EEF0E08081A4
:103990008460808378940C94DC218CE091E00C941A
:1039A000EA188091C0028530A9F48091C002853068
:1039B00079F40E94711A8091BE028823B1F30E94AB
:1039C000321A882391F30E94471D0E944B07EDCFC6
:1039D0000C949C1A089508950C94EE1C292F3327FB
:1039E00023303105C9F060F42130310581F02230F7
:1039F000310509F044C08BE390E028EA32E043C08F
:103A000021323105E1F02232310549F138C082E13D
:103A100090E023EE32E037C099278130910549F0DC
:103A200028F0029761F5E2E8F2E005C0E4EAF2E08E
:103A300002C0E4E9F2E0849190E09F0124C06115A6
:103A4000710541F061307105D1F489E090E023ED1A
:103A500032E019C089E090E02AEB32E014C0611531
:103A6000710541F06130710551F486EB90E025EF6E
:103A700032E009C080E490E02BEA33E004C080E04B
:103A800090E020E030E0FA0131832083089519BCF2
:103A900082E089BD09B400FEFDCF8091D8008F7D02
:103AA0008093D8008091E00082608093E000809154
:103AB000E00081FDFCCF0895CF92DF92EF92FF925C
:103AC0000F931F93CF93DF93EC018B017A010E9438
:103AD000BA1E811133C0E114F10439F0F70180817D
:103AE0009181081B190BC80FD91FC12CD12C0115AE
:103AF000110519F18091E80085FD16C08091E8005C
:103B00008E778093E800E114F10449F0F701808199
:103B10009181C80ED91ED182C08285E00FC00E945B
:103B2000BA1E882321F30AC089918093F1000150C5
:103B30001109FFEFCF1ADF0ADACF80E0DF91CF91D2
:103B40001F910F91FF90EF90DF90CF9008952091FB
:103B5000C7023091C8022617370748F06115710572
:103B600039F42091E8002E772093E80001C0B901D4
:103B7000FC0120E06115710579F18091C002882374
:103B8000F1F18530F1F18091E80083FD3CC0809136
:103B9000E80082FD2EC08091E80080FFEBCF2091ED
:103BA000F3008091F20090E0922B6115710551F0C5
:103BB0008830910538F421912093F100615071090A
:103BC0000196F3CF21E0089709F020E08091E8000A
:103BD0008E778093E800CECF2111CFCF0AC080919D
:103BE000C002882361F0853061F08091E80083FD98
:103BF0000AC08091E80082FFF2CF80E0089582E061
:103C0000089583E0089581E008952091C7023091DE
:103C1000C8022617370748F06115710539F420915D
:103C2000E8002E772093E80001C0B901FC0120E0F4
:103C30006115710591F18091C002882309F440C09B
:103C4000853009F43FC08091E80083FD3DC080913C
:103C5000E80082FD2FC08091E80080FFE9CF20912D
:103C6000F3008091F20090E0922B6115710559F0FC
:103C70008830910540F424912093F10031966150F1
:103C800071090196F2CF21E0089709F020E08091B8
:103C9000E8008E778093E800CBCF2111CCCF0AC00B
:103CA0008091C002882361F0853061F08091E80046
:103CB00083FD0AC08091E80082FFF2CF80E0089582
:103CC00082E0089583E0089581E00895982F973069
:103CD00068F59093E900981739F07091EC00209105
:103CE000ED005091F00003C0242F762F50E021FD0D
:103CF00002C09F5FECCF3091EB003E7F3093EB0032
:103D00003091ED003D7F3093ED003091EB0031605C
:103D10003093EB007093EC002093ED005093F00093
:103D20002091EE0027FDE5CF80E008958F7080930D
:103D3000E90081E008958091C10287FF11C0809160
:103D4000E80082FD05C08091C0028111F8CF11C04A
:103D50008091E8008B770BC08091C002882349F0E6
:103D60008091E80080FFF8CF8091E8008E77809303
:103D7000E80008952091E4003091E50095E6409137
:103D8000EC00842F817040FF23C08091E80080FD0B
:103D90001DC08091C002882399F0853099F08091F0
:103DA000EB0085FD11C04091E4005091E50024171F
:103DB000350729F3915011F09A01E1CF84E008957D
:103DC00082E0089583E0089581E0089580E00895F9
:103DD0004091E80042FFDDCF08950E945B1F0E94E2
:103DE000631FE0EEF0E0808181608083E8EDF0E029
:103DF00080818F77808319BCA7EDB0E08C918E7F96
:103E00008C9380818F7E80831092BF0208950F93E0
:103E10001F93CF93DF930E945B1F0E94631FC8ED27
:103E2000D0E088818F7788838881806888838881C3
:103E30008F7D888319BC1092C0021092BC02109230
:103E4000BE021092BD0200EE10E0F80180818B7F6F
:103E5000808388818160888342E060E080E00E9406
:103E6000661EE1EEF0E080818E7F8083E2EEF0E07E
:103E7000808181608083808188608083F801808177
:103E80008E7F8083888180618883DF91CF911F91AD
:103E90000F910895E8EDF0E080818F7E8083E7ED5B
:103EA000F0E080818160808384E082BF81E0809344
:103EB000BF020C94071FE8EDF0E080818E7F8083C5
:103EC0001092E20008951092DA001092E100089535
:103ED0001F920F920FB60F9211242F933F934F937F
:103EE0005F936F937F938F939F93AF93BF93EF9362
:103EF000FF938091E10082FF0BC08091E20082FF7E
:103F000007C08091E1008B7F8093E1000E94DB215C
:103F10008091DA0080FF1DC08091D80080FF19C019
:103F20008091DA008E7F8093DA008091D90019BCED
:103F300080FF0BC082E089BD09B400FEFDCF81E0A7
:103F40008093C0020E94B11B04C01092C0020E9464
:103F5000BF1B8091E10080FF19C08091E20080FFCB
:103F600015C08091E2008E7F8093E2008091E20094
:103F700080618093E2008091D80080628093D800B5
:103F800019BC85E08093C0020E94C41B8091E100AF
:103F900084FF2FC08091E20084FF2BC019BC82E017
:103FA00089BD09B400FEFDCF8091D8008F7D80933C
:103FB000D8008091E1008F7E8093E1008091E20043
:103FC0008F7E8093E2008091E20081608093E20026
:103FD0008091BC02882311F084E007C08091E30047
:103FE00087FD02C081E001C083E08093C0020E948F
:103FF000CC1B8091E10083FF29C08091E20083FF08
:1040000025C08091E100877F8093E10082E080936A
:10401000C0021092BC028091E1008E7F8093E1008B
:104020008091E2008E7F8093E2008091E2008061C7
:104030008093E20042E060E080E00E94661E809192
:10404000F00088608093F0000E94C21BFF91EF9106
:10405000BF91AF919F918F917F916F915F914F91A0
:104060003F912F910F900FBE0F901F9018951F92A8
:104070000F920FB60F9211242F933F934F935F939C
:104080006F937F938F939F93AF93BF93CF93DF9360
:10409000EF93FF93C091E900CF708091EC00D82F8F
:1040A000D17080FDD0E81092E9008091F000877F08
:1040B0008093F00078940E947B201092E900809118
:1040C000F00088608093F000CD2BCF70C093E900A2
:1040D000FF91EF91DF91CF91BF91AF919F918F9120
:1040E0007F916F915F914F913F912F910F900FBEF4
:1040F0000F901F9018951F93CF93DF93CDB7DEB726
:10410000AA970FB6F894DEBF0FBECDBFE1ECF2E088
:104110008091F100819322E0E93CF207C9F70E9407
:10412000EA1B8091E80083FF2EC18091C10290912B
:10413000C202492F50E04A30510508F024C1FA016B
:10414000EF55FF4F0C940B22803821F0823809F094
:104150001AC108C08091BD029091BE02992389F0D6
:1041600082600FC08091C5028F70873008F00BC14C
:104170008093E9008091EB0085FB882780F91092FD
:10418000E9009091E800977F9093E8008093F10018
:104190001092F100D1C0282F2D7F09F0F4C08823A0
:1041A00019F0823061F0EFC08091C302813009F0D4
:1041B000EAC0933009F080E08093BE022EC0809167
:1041C000C30281112AC08091C5028F702FEF280F82
:1041D000263008F0D8C08093E9002091EB0020FF42
:1041E0001CC0933021F48091EB00806214C0909148
:1041F000EB0090619093EB0021E030E0A90102C058
:10420000440F551F8A95E2F74093EA001092EA00A6
:104210008091EB0088608093EB001092E900809120
:10422000E800877F8093E8000E949B1EACC081114C
:10423000AAC01091C3021F778091E3008078812B80
:104240008093E3008091E800877F8093E8000E94DC
:104250009B1E8091E80080FFFCCF8091E300806886
:104260008093E300111102C082E001C083E08093DB
:10427000C00289C08058823008F085C08091C30296
:104280009091C4028C3D53E0950779F583E08A83D1
:104290008AE289834FB7F894DE01139620E03EE06E
:1042A00051E2E32FF0E050935700E49120FF03C068
:1042B000E295EF703F5FEF708E2F90E0EA3010F0E4
:1042C000C79601C0C0968D939D932F5F243149F707
:1042D0004FBF8091E800877F8093E8006AE270E03A
:1042E000CE0101960E94A71D16C06091C502709173
:1042F000C602AE014F5F5F4F0E94EC1CBC01892BD0
:1043000009F441C09091E800977F9093E80089817B
:104310009A810E94051E8091E8008B778093E800C7
:1043200032C0803881F58091E800877F8093E80073
:104330008091BC028093F1008091E8008E7772CF6B
:10434000811121C08091C3029091C40299270297E4
:10435000D4F48091E800877F8093E8008091C302C5
:104360008093BC020E949B1E8091BC02811106C0FA
:104370008091E30087FD02C081E001C084E080936A
:10438000C0020E94D61B8091E80083FF0AC0809182
:10439000E800877F8093E8008091EB008062809343
:1043A000EB00AA960FB6F894DEBF0FBECDBFDF912B
:1043B000CF911F9108950895CF938091C0028823D3
:1043C000A1F0C091E900CF709091EC00892F81702D
:1043D00090FD80E8C82B1092E9008091E80083FDF1
:1043E0000E947B20CF70C093E900CF91089597FB86
:1043F000072E16F4009407D077FD09D00E941122F1
:1044000007FC05D03EF4909581959F4F08957095D7
:1044100061957F4F0895EE0FFF1F0590F491E02DF9
:104420000994AA1BBB1B51E107C0AA1FBB1FA617FB
:10443000B70710F0A61BB70B881F991F5A95A9F74D
:1044400080959095BC01CD010895FB01DC0104C06D
:104450008D910190801921F441505040C8F7881B7C
:10446000990B0895F999FECF92BD81BDF89A9927CD
:1044700080B50895A8E1B0E042E050E00C946622D7
:10448000262FF999FECF92BD81BDF89A019700B40D
:10449000021639F01FBA20BD0FB6F894FA9AF99AAD
:1044A0000FBE08950396272F0E9441220E944022AA
:1044B000252F0E944122242F0C9441220196272F60
:1044C0000E9441220C944022DC01CB01FC01F999AD
:1044D000FECF06C0F2BDE1BDF89A319600B40D9250
:0C44E00041505040B8F70895F894FFCF09
:1044EC00C8002802280850011E0A14011A1B3D1B83
:1044FC001E1BAD1BA91B1D1B01E200E900EA00B548
:10450C0000B600B700CD008301CC008A0192019463
:10451C00012102230224022502260227022A02B3C9
:10452C0000B4006F007000818283E200E900EA00B1
:10453C00B500B600B700CD008301CC008A01920112
:10454C0094012102230224022502260227022A02B8
:10455C00B300B4006F00700081828367313233374F
:10456C0090919293959496973435F1F0F6F5F4007A
:00000001FF
